:020000040000FA
:060000000219FD02031CC1
:03000B0002008D63
:03001300020535AE
:03001B0002009050
:03002B000202D1FD
:03005B0002054457
:030073000203097C
:100080000406080C10182030406080A0C0054032E3
:10009000C2AFC2A853E6EFC28E856B8BC0D0D2D35D
:1000A000C0E0C0F0C2CAA8CCA9CDD2CAD2AF758A6E
:1000B00000C3E8956CF8E9956DF9C3E913F9E81305
:1000C000F8E5666007C3E913F9E813F8E97025E875
:1000D000956E4020956E501CE582B410177C007B15
:1000E000007A007908900000A86AE5667004C3E809
:1000F00013F801FD900000D2A8D2AA61E7E0FDC389
:100100009CC39840EF98EB33FB0582E0FCC39DC392
:100110009840E198EB33FB0582E0FDC39CC3984017
:10012000D398EB33FB0582E0FCC39DC39840C59890
:10013000EB33FB0582E0FDC39CC39840B798EB33DB
:10014000FB0582E0FCC39DC39840A998EB33FB05F7
:1001500082E0FDC39CC398409B98EB33FB0582E093
:10016000FCC39DC398408D98EB33FB0582217890AA
:100170000000D2A8D2AA61E7E0FDC39CC39840EF7B
:1001800098EA33FA0582E0FCC39DC39840E198EAFF
:1001900033FA0582E0FDC39CC39840D398EA33FA52
:1001A0000582E0FCC39DC39840C598EA33FA0582F6
:1001B000E0FDC39CC39840B798EA33FA0582E0FC9F
:1001C000C39DC39840A998EA33FA0582E0FDC39C19
:1001D000C398409B98EA33FA0582E0FCC39DC3981C
:1001E000408D98EA33FA0582EBC46B6A54F0F9EA61
:1001F000C454F0C3996009900000D2A8D2AA61E764
:10020000EBF4C454F0F9EAF4C4540F49FAEBF4C423
:10021000540FFBC3EAF99460FAEB9400FB5020C33F
:10022000E97B007A0079006016C3135006F9C39584
:1002300052600AE9F5527553007900800205533087
:100240003A27C3EA94D0F8EB9407F9400BE8FAE9AF
:10025000FB203509D235415D303502C235203902E7
:10026000B235C3EA33FAEB33FBEB2B3B3BF9C3EB81
:1002700013FBEA13FAEA29FAEB3400FB30E3047AC1
:10028000FF7BFFE5255403601B202A18E55D33F949
:10029000EB7007C3E99A4002E9FAE53CC4332AFA55
:1002A000EB3400FBC3EA33C4540FF8EB33C454F00F
:1002B00048F87005EA60027801900000D2A8D2AA3E
:1002C000E5226002152281D4900000D2A8D2AA6152
:1002D000E7C0D0C0E0C2CF0541E5666009E56560D2
:1002E000057565006104756501E52360021523C38A
:1002F000E55460057555006104E5552401F5555038
:10030000037555FFD0E0D0D032C2AF53E67F75926F
:10031000FA7593FFC22053917FD2AF32C0E0E58AD5
:10032000303408856B8BF0A3D0E032D0E0C2AF53FD
:10033000E6EFC0D0C0E0C0F0D2D3D2AF5388EFA870
:100340008AA98CAA40308D010A758A00758C0075C7
:100350004000438810E566700AC3E833F8E933F9D2
:10036000EA33FA30331FE8C4540FFAE9C454F04AB0
:10037000FAC3132AFAC3E833F8E933F9E82AFAE9A9
:100380003406FB61D830320FC3E833E933FAE82A88
:10039000FAE93400FB61D8303115E875F056A4AAAB
:1003A000F0E975F056A42AFAC5F03400FB61D8C311
:1003B000EA13FAE913F9E813F8E875F056A4AAF07D
:1003C000E975F056A42AFAC5F03400C313FBEA130A
:1003D000FAC3EB13FBEA13FAC3EB94125009C3EA16
:1003E0009434EB940750160522E52270021522C3BF
:1003F000E52294325002A128755400A12BE5226019
:100400000215223036067C007D088117AC31AD32F2
:10041000303A04AC33AD34C3EA9CFAEB9DFB92084E
:10042000AE60AF61303A425007203509D235813590
:10043000303502C235303504AE62AF63203902B2C6
:1004400035C3EA33FAEB33FBA208500AEAF424017D
:10045000FAEBF43400FBC3EA9450FAEB9400FB503F
:100460001478007A007B008175A208500878007A21
:10047000007B0081D4E5255403601B202A18E55D2C
:1004800033F9EB7007C3E99A4002E9FAE53CC4335B
:100490002AFAEB3400FBEA8EF0A4F9AAF0EB8EF016
:1004A000A42AFAC5F03400FBC3EB13FDEA13F8C32A
:1004B000ED13FDE813F80FEF146004C3E833F8C33D
:1004C000E933EA33FAEB33FBDFEDEB30E30678FF99
:1004D0007AFF7B078854D230E86003755500C3E586
:1004E0005BFC955C4002AC5CC3EC95545008EC7529
:1004F000F008A4FAABF0EAF4F8EBF45407F9C3E817
:10050000948CFAE99400FB50047A007B00885689A9
:10051000578A588B5975230AD0F0D0E0D0D053F7C2
:10052000DF43F74043E6103275230AD0F0D0E0D025
:10053000D043E61032C2AAD28EC2CA85CC6C85CD19
:100540006DD2CA32C2AFC0D0C0E0D2D3A8F9E55A4A
:1005500030E20AE5FA20E23520E132A165E5FA3021
:10056000E22B20E128C3E55713F8E55613F5E98897
:10057000EAC3E55913F8E55813F5FB88FC85575A8B
:1005800053F7BFD2A8303402D2AA53E6EF53F7DFB5
:10059000D0E0D0D0D2AF32790180147903801079C5
:1005A0000A800C791E80087964800479C8800078FC
:1005B00017E4D5E0FDD8FAD9F62278FF202828796B
:1005C000A1E76023E548601F74FF8548F084853FFC
:1005D000F030290375F005A4F8C5F0600278FFC378
:1005E000E8955D5002A85D885C22C3E54794A0E5CC
:1005F000489400E55C500314A1FB046002F55C2202
:1006000075E89022055EC3E55E9408405330EDF432
:10061000A8BDA9BE755E00E9FA79A0E76041EA705D
:1006200006E55F6018800CC3E8955F600EE55F50DB
:1006300005600A1480070460FA8002E55FF55FC375
:100640009569401B755BC0C394044013755B80C300
:100650009404400B755B40C394044003755B002217
:10066000E55B2410500274FFF55B22743279A68793
:10067000F0A4C5F0A2F733F55D227547007548F088
:1006800022C2AFC2CAA8CCA9CDAA4130CF010AD29A
:10069000CAD2AFC3EA13FAE913F9E813F8AB42ACD4
:1006A0004388428943C3E89BF8E99C20280A547F89
:1006B000F9302C02E19FC1F8AD448A44F9EA9D5417
:1006C0007FFA600678FF79FFC1DDAE45AF468B4506
:1006D0008C46A842A943C3E89EF8E99FF9C3E548C0
:1006E00013FBE54713FAE82AF547E93BF5485006BE
:1006F0007547FF7548FFE145AA47AB48AC47AD4891
:100700007E047F02C3EB9404400D1E1FC3EB9408CC
:1007100040052029021E1FC3ED13FDEC13FCDEF77C
:10072000C3EA9CFAEB9DFBEF6009C3E913F9E813F8
:10073000F8DFF7EA28FAEB39FB8A478B4850067B4B
:10074000FF8B478B48C3EB94025002D22C30280415
:100750007F03E1707892E6FFC3E53D948240110F7C
:10076000C3E53D94A040010FC3EF940640027F050E
:100770007E02E548C4540FF9E548C454F0F8E54753
:10078000C4540F28F8C3E89EFAE99400FB4009C35B
:10079000EA9401EB940050047A01E4FB0207EBAA0F
:1007A00047AB48EBC4FEEAC4540F4EFCC3EA9CFAC4
:1007B000EB9400FBC3E813C313F8EA28FAEB340008
:1007C000FB8A478B48C3EB94024002C22C7802EBB1
:1007D000C4FE7B00EAC4540F4EFAC3EA98FA4005FF
:1007E000C3940150027A017892E6FF302002E1EBD7
:1007F000854E92854F93D22043E680C3E49AF8E475
:100800009BF9C3E833F8E933F9302C03020880E898
:10081000FAE9FBD3E913FDE813FC884E894FC3EFD7
:1008200094036038EF20E00CE82CF8E93DF9ECFA8D
:10083000EDFB8013E828F8E939F9C3E82401F8E969
:100840003400F97AFF7BFFC3EF9403400F8A508B8B
:1008500051884A894B8C4C8D4D0208B5885089517E
:100860008A4A8B4B8C4C8D4D3028127550F0755147
:10087000FF754CF0754DFF754EF0754FFF0208B5D2
:10088000E8FAD3E813FC884EC3EF94036021EF200D
:10089000E007E82CF8ECFA01A0E8282401F87AFF38
:1008A000C3EF940340098A50884A8C4C0208B588EB
:1008B000508A4A8C4C30200201B5753A02D220434E
:1008C000E680E5255403602DA847A948C3E913F93C
:1008D000E813F8302804E92440F9C2AF53E67F75E5
:1008E0009100C3E498F594E499F595759104D220AC
:1008F00043E680D2AF22D221754900752000302B0B
:10090000037520402114D221754900752040302BF9
:100910000375200078017901202C20E5255403601F
:1009200002C2217914E548C313700104F8C394147A
:1009300040027814302804781B791BC3E833F8C3CD
:10094000E933F9202010E549600C302803D53A043A
:10095000D22221C711BD0549E59B5440B520022193
:10096000B130280908C3E899400118214320210A21
:1009700008C3E899400221142143C22153E67F7540
:100980009100302C117594007595F0759104D2206A
:1009900043E680020914E5487EFFC3334009C333B0
:1009A0004005C3334001FEC3E49E759400F59521D4
:1009B0008BC3E5399401500221143021022114D84F
:1009C0000221C52143C222C2AF53E67F7591008543
:1009D0005094855195759104854A92854B93D22008
:1009E00043E680D2AFE5255403600720290205398C
:1009F000801030220D202B0A20210715811581023D
:100A000013FC2278003021027801E53D75F007A43F
:100A1000F9E5F028F5F0E9A2F013A2F113A2F21320
:100A2000F53DC394785003753D78C3E53D953E4050
:100A30000CC296C294C29075D4FF75D57F30200247
:100A4000413D854C92854D93D22043E6802220384B
:100A500013C2AFC291D29575D47F75D57ED2AF75D2
:100A60009F126142C2AFC291D28775D4FF75D51F64
:100A7000D2AF759F126142203813C2AFC29075D4B5
:100A8000FF75D56DD295D2AF759F326142C2AFC2AC
:100A90009675D4FF75D56DD287D2AF759F0261422E
:100AA000203813C2AFC295D28775D4FF75D56DD2E9
:100AB000AF759F026142C2AFC287D29575D4FF75F0
:100AC000D56DD2AF759F328079203813C2AFC294F2
:100AD00075D4FF75D51FD287D2AF759F128063C2C0
:100AE000AFC29475D47F75D57ED295D2AF759F1263
:100AF0008050203813C2AFC287D29175D4FF75D50C
:100B00001FD2AF759F32803AC2AFC295D29175D4D1
:100B10007F75D57ED2AF759F028027203813C2AF74
:100B2000C29675D47F75D57ED291D2AF759F028063
:100B300011C2AFC29075D4FF75D51FD291D2AF75D7
:100B40009F32227A147B7880127A107B8C800C7A08
:100B50000D7BB480067A0B7BC88000E564D5E0018C
:100B6000227902E4C291D5E0FDD294D5E0FDC29491
:100B7000D5E0FDD291D5E0FDE920E002D29630E04B
:100B800002D290E564D5E0FDE920E002C29630E0B3
:100B900002C2907496D5E0FDD9C9EAF8D5E0FDD837
:100BA000FBDBB8C29122C296C294C290C295C29198
:100BB000C28775D4FF75D57F22788076FF0876FFCF
:100BC0000876FF0876FF0876FF0876FF08760908A2
:100BD00076FF087601788C76010876FF0876FF08A4
:100BE00076FF0876FF0876FF0876030876FF08761A
:100BF000FF0876FF0876250876D008762808765014
:100C00000876040876FF0876020876FF08767A08E8
:100C100076FF0876070876010876FF0876FF0876E3
:100C20000008760022FA75F00CA4ABF0EAC333F8A2
:100C3000740133F9E8C333F8E933F9E8C32BF8E971
:100C40003400F9E8C333F8E933F9227888E6C3942D
:100C500003D23A5002C23AC238E630E102D238A298
:100C60003892397886E6149000809378A6F67886D4
:100C7000E6F53FC394025003753F02789CE6753E4B
:100C8000FFB40203753EA0B40303753E8278A0E66C
:100C9000F8600674282409D8FCF5697896E6912551
:100CA00088318932789EE69125883389347897E6B1
:100CB00091258835893671A6223036117A007B005D
:100CC0007CFF7D007E00B11F8B618A6022303A225A
:100CD0007896E6FA7B00789EE6FC7D00C3EA33FA5C
:100CE000EB33FBC3EC33FCED33FD7E0AB11F8B63AA
:100CF0008A627896303A02789EE6FA7B007897E628
:100D0000FC7D007E00303A10C3EA33FAEB33FBC3BC
:100D1000EC33FCED33FD7E0AB11F8B618A6022C388
:100D2000EC9EFCED9400FDC3EC9AFCED9BFDC3EC46
:100D30009423ED940050047C237D00C3EC94FFEDDC
:100D4000940140047CFF7D017BFF0B7A000AEA706E
:100D500009C3EC33FCED33FDA14AEC8AF0A4AEF0FC
:100D6000ED8AF0A42E947C40E4EAF460DD22D236D1
:100D700091B91205A31205A37A007B007C1012051D
:100D80009BE5542AFA74003BFBDCF37C04C3EB13B1
:100D9000FBEA13FADCF7FFEB60027FFFC23691B982
:100DA0002278A5E6F954037000E9540C7000E95468
:100DB000307000E954C070002275670075680075D6
:100DC00097DE7597AD7581C043FF8075EF0675A9F5
:100DD0000071A675807F75F1F075A48075807F75B0
:100DE000D4FF75900075F27375A57375900075D575
:100DF0007F75A60175E34075E20271A6E4F8F6D8A6
:100E0000FD71B912144078988664753001C2AF1232
:100E100005AB71431205A371491205A3714F120569
:100E2000A3B1A1C2AF75670075680078FA79FA308E
:100E30008507D9FBD8F7021C00914B91B9789886A9
:100E40006471A675A91375A71075C10075A7007503
:100E5000660075E405758811758E0475890975C875
:100E60000475910475D84075D90875F782759E038D
:100E700075960175DB4275DA4275A82375E69075A3
:100E8000B801759B80759D0075D10C75BCB975BB9B
:100E90001075E88075B201120597D2AF753C00C29B
:100EA000301205ABC231C232C233C2347552007542
:100EB00053007522001205A7C3E522940A5002E1EF
:100EC00089D2317522001205A7C3E522940A500287
:100ED000E189C231D2327522001205A7C3E52294FE
:100EE0000A5002E18975E4D5758851758E017589BE
:100EF000AA758C00758D00C2A9D2ABD2AA756B8081
:100F0000756A14756E50C232D23475220A1205A762
:100F1000756A10C3E522940A755200755300406942
:100F2000758E0C756B00756A28756E2875220A120D
:100F300005A7756A20C3E522940A7552007553000F
:100F40004047758E0C756B80756A14756E1475222A
:100F50000A1205A7756A10C3E522940A7552007536
:100F60005300402575E405758811758E047589094F
:100F7000D2A9C2ABC2AAC234D2337522001205A7CD
:100F8000C3E522940A4002C12312059B20300302CC
:100F90000E23C2AF714371437143D2AF1205AB2030
:100FA0003403303A0302104C12059B788CE6C3944C
:100FB00001500302104CE530C39401500302104C61
:100FC0007567A57568F17F02D23691B91205A7C27F
:100FD000AFC23691B9C3E554947FD2AF406E1205CB
:100FE00097C2AF7155D2AFDFDFB16EC3EF7897F61E
:100FF0001205AB12152D7F0AD23691B91205A7C280
:10100000AFC236120CB9C3E554947FD2AF50E71289
:101010000597C2AF120B4312059F120B43D2AFDFED
:10102000D7120D6EEF24037896F6F87997E7C394FC
:10103000234003985006E824237897F61205AB91D5
:1010400087B15C1205A7120CB9020E2375670075F3
:1010500068001205A7C3E55494014003020F9FC224
:10106000AF120B55120B55120B55D2AF1205AB75C3
:101070003000E4F537F5380537E537F4703F0538CB
:10108000789AE67819146012783214600D787D141D
:10109000600878FA146003753800C3E53898401D7D
:1010A000120BA6120597153875370078998664C219
:1010B000AF120B55D2AF789886641205A712059F20
:1010C000E5237003020E23C3E5549401500AC3E5DF
:1010D00052940150160210771205A7E523700302FF
:1010E0000E2375520075530002128DC3E552940110
:1010F0007017C2AF120BA678998664120B437898CA
:101100008664D2AF1205A7417FC3E55294027017DF
:10111000C2AF120BA678998664120B497898866440
:10112000D2AF1205A7417FC3E55294037017C2AF37
:10113000120BA678998664120B4F78988664D2AF0A
:101140001205A7417FC3E55294047017C2AF120B7A
:10115000A678998664120B5578988664D2AF1205EA
:10116000A7417FC3E55294057017C2AF120BA67852
:10117000998664120B5578988664D2AF1205A74100
:101180007FC3E55294077019C3E5539406500201DA
:10119000C77401303A0274037888F6C238C2394104
:1011A0007FC3E55294087019C3E5539406500201B9
:1011B000C77402303A0274047888F6D238D23941C2
:1011C0007FC3E55294097017C3E55394065002019A
:1011D000C7303A0BC37888E69402F6C23A417FC31F
:1011E000E552940A7016C3E5539406500201C720D5
:1011F0003A0A7888E62402F6D23A417FC3E552944F
:10120000147025C3E5539406500201C7C2AF901A6B
:101210000B740093D2AF7888F613C238C2394002FB
:10122000D2384002D2398057C3E55294157038C382
:10123000E5539406404FC2AF901A0B740093D2AF9F
:10124000F8B801027402B802027401B8030274040F
:10125000B8040274037888F613C238C2394002D247
:10126000384002D2398018C3E552940C701175676A
:10127000A57568F1C3E5539406400A9187D2AF750E
:10128000520075530075670075680001C7C2AF1240
:101290000BA6E4D2AFE4F55EF524F525F53D755EC9
:1012A0000812059712060030EDFDA8BDA9BEE97031
:1012B00001F8885F120604755E08C2AF12066B85DE
:1012C0005D5B855D5CD2AF75A71075C13075A700F9
:1012D00075A903756601303A07C238303502D23835
:1012E000D228753900120AF2120B1B12067A120666
:1012F0008112067A12068112067A120906120A0370
:10130000120A4E1206811208F6202C031205BA307A
:101310002C031205EA120A03120A77120681120937
:1013200006120A03120AA01206811208F6120A0314
:10133000120AC9120681120906120A03120AF212CF
:1013400006811206001208F6120A03120B1B12067F
:1013500004120681302827855D5B79187A0CC3E575
:101360003999400EC228D2298A3B855D5B855D5C38
:10137000800CC3E554940140030212FA8104302921
:101380001F202B1CE53B147006C229D22A41FAF516
:101390003B203A07C3E554940140030212FA8064EB
:1013A000753C00203A0F78FA79A4E760027803C30D
:1013B000E55598504FE523604B303A17203805200B
:1013C0003507800F303502800A202B07D22B855D30
:1013D0005B612A78F0302B05855D5B7820C3E5489A
:1013E0009850030212FA302B1BC22BC23830350240
:1013F000D238D229753B12855D5B41FA053CE55434
:1014000060028107753C00C2AF120BA675240075FF
:10141000250075A91375A71075C10075A70075661D
:1014200000D2AF1205A7120BA678A4E66006D295EB
:10143000D291D287C3E53C94044003020E2301728B
:10144000901A0D782091C0E520B4550AA391C0E50B
:1014500020B4AA0280137567A57568F1120BB991C3
:1014600087756700756800801D901A0378807B0A75
:1014700091C0A308DBFA901A0F788C7B1A91C0A355
:1014800008DBFA901A2922C2AFB10391E0901A004A
:10149000741091C5A3740791C5A3742191C5901AC6
:1014A0000378807B0A91C4A308DBFA901A0F788C2A
:1014B0007B1A91C4A308DBFAB11691F4901A292281
:1014C000E493F622E6438F01538FFDFFC3E5839437
:1014D0001C400122EF8567B78568B7F0538FFE2265
:1014E000438F02438F018567B78568B7901A0DF067
:1014F000538FFC22901A0D745591C5901A0E74AA40
:1015000091C5227A3079D07820901A4091C0E52098
:10151000F709A3DAF7227A3079D0901A40E791C51B
:1015200009A3DAF9227C051205ABDCFB22C2AF125B
:101530000B43120B49120B4F120B5512059F120B46
:1015400043120B49120B4F120B5512059F120B43FE
:10155000120B49120B4F120B55D2AF22C2AF120B16
:1015600055120B4F120B49120B4312059F120B55CC
:10157000120B4F120B49120B4312059F120B5512FF
:0B1580000B4F120B49120B43D2AF229D
:1019FD00020DB9100721FFFFFFFFFFFF09FF01FFD8
:101A0D0055AA01FFFFFFFFFF03FFFFFF25D0285061
:0D1A1D0004FF02FF7AFF0701FFFF0000FF3A
:101A400023565F485F37302320202020202020208D
:101A500023424C48454C492445464D3842323123B7
:101A60002020202020202020202020202020202076
:101C0000C2AFC2D37597DE7597AD7581C075A90057
:101C100043FF80752438752503B1DB7529A5752A26
:101C2000F143F12053A4DFD28575D4FF75E3407DE5
:101C3000FA780379E67C10752200752300901DE880
:101C40007B0675249875250130850281482085081A
:101C5000D8FBD9F9DCF781BA308508D8FBD9F9DC93
:101C6000F781BAB19BE493A3C39A6004DDC381BA40
:101C7000DBDBB18D600281317B08E493FAA3B16EA6
:101C8000DBF87A30B16E752200752300B18DEAFC65
:101C9000EBFDC3ED94FE400EB18D8A278B28ED300D
:101CA000E0048A828B83B18D7AC270D8C3ED94FE32
:101CB000601950CEBD0029EC600F7520007521FF22
:101CC000752900752A000200008100A827A92808AC
:101CD00009D804D90281DDB191EAF281D10D81A642
:101CE000C3ED94035051EDA2E092007AC5C3E582A2
:101CF0009400E583941C508C200010438F02438F86
:101D0000018529B7852AB7F0300027A827A9280818
:101D100009438F01538FFDD804D902A132C3E58353
:101D2000941C4003A3A117E28529B7852AB7F0A325
:101D3000A117538FFC81827AC1BD030CE493A3FAEF
:101D4000B152DCF8B14A81828184AA22AB23B16E00
:101D5000EBFAEA6222752608C3E52313F523E52290
:101D600013F52250066323A0632201D526EAB1DBD6
:101D7000B1DB75260AEAF4200102D285300102C2E5
:101D800085B1DBC3134002C201D526EB22B191EA33
:101D9000FB208502A191308502A196752608AE240C
:101DA000AF25C3EF13FFEE13FEB1DFB1DBC3EA13C0
:101DB0003085024480FA30E703632201C3E5231330
:101DC000F523E52213F52250066323A0632201D5F3
:101DD00026D9E52265236523F52222AE24AF250E00
:101DE0000FDEFEDFFCD20122424C48656C693437BD
:061DF0003164E8B20601B7
:00000001FF
